:020000040000FA
:0A000000000000008FEF00F0A2D016
:08001800EFD0106E960E076E8A
:10002000980E086E55D8D8B4CA90D8A4CA80FC0FD0
:10003000D8A0CA92D8B0CA82800E076E960E086EFB
:10004000980E0B6E0C6ACAB025D8CAB223D842D813
:100050000704CB6E07C009F008C00AF000500D6E0F
:100060000E6E003C0E6A4BD80C50102E0AD0BE6E9D
:100070000C0EBD6E0BBEBD8A0BBCBD889394CA84AA
:100080001200BB6E0C0EBA6E0BBEBA8A0BBCBA88DD
:100090009492F5D700D8D8900B320832073212006C
:1000A0000A6A096EFF0E09260A2200D0D8A01200A3
:1000B000030E086EE60E02D8F5D7086AFE0F076E2B
:1000C000E86A085AD8A012000000070600D0F8D746
:1000D0000C6A0B6A100EF36E08340B360C3609509E
:1000E0000B5C0A500C5805E309500B5E0A500C5A81
:1000F000D88007360836F32EEFD707501200095084
:100100000D02F3CF0BF0F4CF0CF00A500D02F350B8
:100110000C2609500E02F3500C260B5012004F0E05
:10012000AF6E240EAC6E900EAB6E00010F0EC16E62
:10013000070EB46EC69AC70E926EE00E936EC00E96
:10014000946E92809282928494949492DAD0F2A4E3
:1001500003D0F294817A11009EAA19D0060EAB1436
:1001600012E1E2CF49F0E1CF48F04A2A10EE4CF01C
:100170004A50E126000EE222AECFE7FF49C0E2FF7F
:1001800048C0E1FF1100AE50AE50AB98AB881100F3
:100190004A504B5C14E04B2AEACF08F0E9CF07F055
:1001A00000EE4CF04B50E926000EEA22EF50076EAD
:1001B00008C0EAFF07C0E9FFD880120004D0E86851
:1001C000076ED8A0120012004A6A4B6A9D8A9F8A65
:1001D000F28EF28C12009D9A00EE4CF0010EF46E3D
:1001E000F36AF306000EF45AEE6AF450F310F9E1E4
:1001F0004A6A4B6A9D8A1200F29EE0CF58F5D8CF2A
:1002000059F5E8CF5AF5F28E0001A19243C0B3FF31
:1002100042C0B2FF807A80A8472A80A017D082B05F
:1002200013D027C02DF026C02CF0EB0E2C242A6E04
:10023000000E2D202B6E4484898A827094908998B8
:1002400013B002D0010E136E4FD001D0139080A2D4
:1002500017D082A013D027C02BF026C02AF0EB0EB7
:100260002A5C2C6E000E2B582D6E4486898A827073
:100270009490899813B202D0020E136E35D001D03B
:1002800013922950275C0DE12850265C0AE180B8C2
:1002900007D0898A8078929813B402D0040E136E26
:1002A00023D02850265C295027580DE282B009D06F
:1002B000898A82709490899813B603D0080E136EC1
:1002C00013D0899811D02650285C275029580CE269
:1002D00082A009D0898A82709490899813B803D03B
:1002E000100E136E01D08998F29E58C5E0FF59C5D3
:1002F000D8FF5AC5E8FFF28E10009EA8FED7AD6E5B
:100300001200939A8A8A0A0ECBDE939A8A9A80B058
:10031000828880A0829880B2828A80A2829A929AF1
:10032000898A94908B9094968B96929889889396CC
:100330008A9693948A949296899693908A909392AF
:100340008A9293988A9867EC07F08BEC0BF088EC14
:100350000DF0400E416E44944496136A2B682A684F
:100360002D6A2C6AD8902B30276E2A30266E010E0B
:100370003F6E400E406E02EE4CF0D8903F34E926BE
:10038000000EEA22EECF42F0EFCF43F04488476AF6
:10039000006A4C0E0A6E500E096E010E3EDE006AB7
:1003A0004C0E0A6E500E096E020E37DE256A236A65
:1003B00003EE4CF00C0EEE68E82EFDD7246A04DF45
:1003C0000ADFCD6AF294F28A870ED56EB16AA192E5
:1003D000A082B36AB26AD08EA292B10EB16E382AF0
:1003E000E86A38B2010F39B0010806E13970342AE1
:1003F000000E352236223722CBDE146EED0E145C51
:1004000005E3FE0E145C01E2166ACAD114AE37D0C1
:10041000166A8C0E145C05E114C016F01768186893
:100420002DD09C0E145C05E114C016F019681A68F2
:1004300025D0AC0E145C05E114C016F01B681C68D6
:100440001DD0BC0E145C05E114C016F01D681E68BA
:1004500015D0CC0E145C04E114C016F01F680ED049
:10046000DC0E145C04E114C016F0206807D0EC0E1A
:10047000145C04E114C016F02168226891D1165270
:1004800003E186EF04F08CD18C0E165CD8A459D011
:10049000172803E114C017F053D014C018F0250E2C
:1004A000175C06E127C029F026C028F0259447D024
:1004B000270E175C06E127C029F026C028F0259AF0
:1004C0003ED0290E175C06E127C029F026C028F08F
:1004D000259C35D0540E175C0AE1006A4C0E0A6E5A
:1004E000500E096E010E0DEC00F0259628D0550E29
:1004F000175C0AE1006A4C0E0A6E500E096E020E7D
:100500000DEC00F025981BD0560E175C0BE18A9677
:100510002390259003014F694E694D694C69448AC7
:1005200000010DD0570E175C09E18A9423922592A1
:1005300003015369526951695069448A000117687F
:100540002FD19C0E165CD8A4F1D0192803E114C059
:1005500019F0EBD014C01AF01A52D8A451D0250EBD
:10056000195C06E127C029F026C028F0259447D061
:10057000270E195C06E127C029F026C028F0259A2D
:100580003ED0290E195C06E127C029F026C028F0CC
:10059000259C35D0540E195C0AE1006A4C0E0A6E97
:1005A000500E096E010E0DEC00F0259628D0550E68
:1005B000195C0AE1006A4C0E0A6E500E096E020EBA
:1005C0000DEC00F025981BD0560E195C0BE18A96B5
:1005D0002390259003014F694E694D694C69448A07
:1005E00000010DD0570E195C09E18A9423922592DF
:1005F00003015369526951695069448A000195D0D9
:10060000250E195C04E11AC040F025848DD0270E18
:10061000195C06E11AC040F0296A286A258A84D04C
:10062000290E195C06E11AC040F029682868258C5B
:100630007BD0540E195C0DE124A00AD01AC000F042
:100640004C0E0A6E500E096E010E0DEC00F0258660
:100650006BD0550E195C0DE124A00AD01AC000F031
:100660004C0E0A6E500E096E020E0DEC00F025883D
:100670005BD0560E195C2BE12F6A1AC02EF08A86C9
:10068000325202E0258001D0259003EE58F0D89038
:100690002E34E926000EEA22EECF05F0EFCF06F069
:1006A00005503424016E06503520026E000E3620AF
:1006B000036E000E3720046E04C04FF303C04EF3E8
:1006C00002C04DF301C04CF32380448A2DD0570E55
:1006D000195C2AE1316A1AC030F08A84325202E091
:1006E000258201D0259203EE58F0D8903034E926C7
:1006F000000EEA22EECF05F0EFCF06F005503424CD
:10070000016E06503520026E000E3620036E000E7C
:100710003720046E04C053F303C052F302C051F3F8
:1007200001C050F32382448A19683AD0AC0E165C9B
:100730000AE11B2803E114C01BF004D014C01CF014
:1007400026EC06F02DD0BC0E165C0AE11D2803E154
:1007500014C01DF004D014C01EF0B0EC06F020D080
:10076000CC0E165C07E11F2804E114C01FF08DECCD
:1007700006F016D0DC0E165C07E1202804E114C058
:1007800020F0AEEC06F00CD0EC0E165C09E121284E
:1007900003E114C021F004D014C022F08FEC06F065
:1007A0001352D8B4B1D0B190010E3F6E4EC242F098
:1007B0004FC243F0010E135C28E1030E2C24286E77
:1007C000000E2D20296E400E406E01EE4CF0D890A8
:1007D0004134E926000EEA22EECF05F0EFCF06F015
:1007E00005503424016E06503520026E000E36206E
:1007F000036E000E3720046E04C057F303C056F397
:1008000002C055F301C054F37CD0020E135C28E102
:10081000030E2A5C286E000E2B58296E400E406E87
:1008200001EE4CF0D8904134E926000EEA22EECFDA
:1008300005F0EFCF06F005503424016E0650352048
:10084000026E000E3620036E000E3720046E04C0C8
:1008500057F303C056F302C055F301C054F351D00F
:10086000040E135C09E13FC040F00301576956696B
:1008700055695469000145D0080E135C20E101EE72
:100880004CF0D8904134E926000EEA22EECF05F074
:10089000EFCF06F005503424016E06503520026E6D
:1008A000000E3620036E000E3720046E04C057F38E
:1008B00003C056F302C055F301C054F322D0100E0A
:1008C000135C1FE101EE4CF0D8904134E926000E94
:1008D000EA22EECF05F0EFCF06F005503424016E8A
:1008E00006503520026E000E3620036E000E3720B3
:1008F000046E04C057F303C056F302C055F301C0A1
:1009000054F3136AB180448A44BA65D9030E3E5C3D
:10091000D8B039D13A50345C3B5035583C503658F9
:100920003D503758D8A021D13D8E3E52D8A451D049
:1009300025B009D023908A9603014F694E694D690D
:100940004C69000145D023A022D08A9604EE58F0CD
:10095000D8903234E926000EEA22EECF05F0EFCF30
:1009600006F005503424016E06503520026E000E4C
:100970003620036E000E3720046E04C04FF303C010
:100980004EF302C04DF301C04CF3239021D08A8670
:1009900003EE58F0D8902E34E926000EEA22EECF6E
:1009A00005F0EFCF06F005503424016E06503520D7
:1009B000026E000E3620036E000E3720046E04C057
:1009C0004FF303C04EF302C04DF301C04CF323803C
:1009D000CBD0010E3E5CD8A451D025B209D02392D1
:1009E0008A9403015369526951695069000145D0E5
:1009F00023A222D08A9404EE58F0D8903334E9260A
:100A0000000EEA22EECF05F0EFCF06F005503424B9
:100A1000016E06503520026E000E3620036E000E69
:100A20003720046E04C053F303C052F302C051F3E5
:100A300001C050F3239221D08A8403EE58F0D8905D
:100A40003034E926000EEA22EECF05F0EFCF06F0B3
:100A500005503424016E06503520026E000E3620FB
:100A6000036E000E3720046E04C053F303C052F32C
:100A700002C051F301C050F3238276D0020E3E5CD7
:100A8000D8A472D03F50405C12E103015769566907
:100A90005569546902EE4CF0D8903F34E926000EB7
:100AA000EA22EECF42F0EFCF43F000015DD040509C
:100AB0003F5C2CE23F2A02EE4CF0D8903F34E9260E
:100AC000000EEA22EECF42F0EFCF43F001EE4CF001
:100AD000D8904134E926000EEA22EECF05F0EFCFA0
:100AE00006F005503424016E06503520026E000ECB
:100AF0003620036E000E3720046E04C057F303C087
:100B000056F302C055F301C054F32ED03F50405C61
:100B10002BE23F0602EE4CF0D8903F34E926000E5F
:100B2000EA22EECF42F0EFCF43F001EE4CF0D89046
:100B30004134E926000EEA22EECF05F0EFCF06F0B1
:100B400005503424016E06503520026E000E36200A
:100B5000036E000E3720046E04C057F303C056F333
:100B600002C055F301C054F336D837AE0BD0376A04
:100B7000366A356A346A256A03EE4CF00C0EEE686C
:100B8000E82EFDD706D037AE04D0376A366A356A0C
:100B9000346A80B410D044A80DD04498476A80B815
:100BA00009D082B004D02606000E275A02D0264A69
:100BB000272A00D005D0650E475C02E34488476AC7
:100BC00080B0828880A0829880B2828A80A2829A35
:100BD0008170EFEF01F03E683D8E156A030E155CE3
:100BE00033E2D8901534E96EEA6AEA36E936EA3635
:100BF0004C0EE926030EEA22EFCF01F0ECCF02F013
:100C0000ECCF03F0ECCF04F03A50015C3B500258BB
:100C10003C5003583D50045815E2D8901534E96E05
:100C2000EA6AEA36E936EA364C0EE926030EEA228B
:100C3000EFCF3AF0ECCF3BF0ECCF3CF0ECCF3DF017
:100C400015C03EF0152ACAE3449A1200250E1B5C1B
:100C500006E0270E1B5C03E0290E1B5C33E180B825
:100C600030D01CC040F040503F5C2BE002EE4CF016
:100C7000D8903F34E926000EEA22EECF42F0EFCFC3
:100C800043F001EE4CF0D8904134E926000EEA2200
:100C9000EECF05F0EFCF06F005503424016E06507C
:100CA0003520026E000E3620036E000E3720046ED3
:100CB00004C057F303C056F302C055F301C054F308
:100CC000448A29D0540E1B5C0CE125A609D01CC017
:100CD00000F04C0E0A6E500E096E010E0DEC00F085
:100CE0001AD0550E1B5C0CE125A809D01CC000F0E1
:100CF0004C0E0A6E500E096E020E0DEC00F00BD079
:100D0000560E1B5C03E11CC032F005D0570E1B5C75
:100D100002E11CC033F01B6812001F68120044A4DB
:100D20001AD044A218D0D8902230466E456A453277
:100D300021504526000E4622465203E1E90E455C4D
:100D400003E3466AE80E456E000145502C24286EE8
:100D500046502D20296E216822681200206812005A
:100D60001E0E1D5C05E11CC032F01CC033F06FD0BC
:100D70002D0E1D5C09E1400E1E5C03E2448044928E
:100D800002D04490448263D02E0E1D5C03E11EC04D
:100D900041F05DD0420E1D5C34E11E5203E124900F
:100DA00058D82ED02480B18044B42AD0136A296A3E
:100DB000286A010E3F6E480E406E4EC242F04FC28E
:100DC00043F0CCC105F0CDC106F005503424016ECE
:100DD00006503520026E000E3620036E000E3720BE
:100DE000046E04C057F303C056F302C055F301C0AC
:100DF00054F3929A898A94908B9092988998448A15
:100E000026D07B0E1D5C22E1256A448A006A4C0EC6
:100E10000A6E500E096E010E0DEC00F0006A4C0EC9
:100E20000A6E500E096E020E0DEC00F003015769B8
:100E30005669556954699298898827C029F026C057
:100E400028F0010E3F6E406E8A968A9400011D685C
:100E50001200B190136A236A256A448A27C029F0D8
:100E600026C028F02F6A2E6A316A306A326A336AE5
:100E700092988988006A4C0E0A6E500E096E010E17
:100E80000DEC00F0006A4C0E0A6E500E096E020E58
:100E90000DEC00F044804492400E416E030157690E
:100EA000566955695469010E3F6E406E02EE4CF072
:100EB000D8903F34E926000EEA22EECF42F0EFCF81
:100EC00043F08A968A94246A476A0001120004015A
:100ED000596958695C0E5B6F7A0E5A6F590E5D6FD7
:100EE000850E5C6F580E5F6F140E5E6F560E616F4D
:100EF000A90E606F550E636F430E626F530E656FE0
:100F0000E30E646F520E676F890E666F510E696F44
:100F1000350E686F4F0E6B6FE60E6A6F4E0E6D6F7B
:100F20009C0E6C6F4D0E6F6F580E6E6F4C0E716F86
:100F3000190E706F4A0E736FDF0E726F490E756F68
:100F4000AA0E746F480E776F7A0E766F470E796F20
:100F50004F0E786F460E7B6F290E7A6F450E7D6FB0
:100F6000080E7C6F430E7F6FEB0E7E6F420E816F1B
:100F7000D30E806F410E836FBF0E826F400E856F60
:100F8000B00E846F3F0E876FA50E866F3E0E896F81
:100F90009E0E886F3D0E8B6F9C0E8A6F3C0E8D6F80
:100FA0009E0E8C6F3B0E8F6FA40E8E6F3A0E916F5C
:100FB000AE0E906F390E936FBC0E926F380E956F18
:100FC000CE0E946F370E976FE30E966F360E996FB5
:100FD000FD0E986F360E9B6F1A0E9A6F350E9D6F31
:100FE0003B0E9C6F340E9F6F5F0E9E6F330EA16F92
:100FF000870EA06F320EA36FB20EA26F310EA56FD7
:10100000E10EA46F310EA76F140EA66F300EA96FFC
:10101000490EA86F2F0EAB6F820EAA6F2E0EAD6F0A
:10102000BE0EAC6F2D0EAF6FFD0EAE6F2D0EB16FFD
:101030003F0EB06F2C0EB36F850EB26F2B0EB56FD7
:10104000CD0EB46F2B0EB76F180EB66F2A0EB96F98
:10105000670EB86F290EBB6FB80EBA6F290EBD6F41
:101060000C0EBC6F280EBF6F620EBE6F270EC16FD5
:10107000BC0EC06F270EC36F180EC26F260EC56F51
:10108000760EC46F250EC76FD80EC66F250EC96FBA
:101090003C0EC86F240ECB6FA20ECA6F240ECD6F0C
:1010A0000B0ECC6F230ECF6F760ECE6F220ED16F4C
:1010B000E40ED06F220ED36F540ED26F210ED56F77
:1010C000C60ED46F210ED76F3B0ED66F200ED96F90
:1010D000B20ED86F200EDB6F2B0EDA6F1F0EDD6F96
:1010E000A60EDC6F1F0EDF6F240EDE6F1E0EE16F8B
:1010F000A30EE06F1E0EE36F250EE26F1D0EE56F6F
:10110000A90EE46F1D0EE76F2E0EE66F1C0EE96F41
:10111000B60EE86F1C0EEB6F3F0EEA6F1B0EED6F05
:10112000CB0EEC6F1B0EEF6F580EEE6F1A0EF16FB9
:10113000E80EF06F1A0EF36F790EF26F1A0EF56F5C
:101140000B0EF46F190EF76FA00EF66F190EF96FF4
:10115000360EF86F180EFB6FCE0EFA6F180EFD6F7D
:10116000680EFC6F180EFF6F030EFE6F170E050161
:10117000016FA00E006F170E036F3F0E026F160E69
:10118000056FDF0E046F160E076F800E066F160ECA
:10119000096F240E086F150E0B6FC80E0A6F150E1F
:1011A0000D6F6E0E0C6F150E0F6F160E0E6F140E68
:1011B000116FBF0E106F140E136F690E126F140EA5
:1011C000156F150E146F130E176FC20E166F130ED8
:1011D000196F710E186F130E1B6F210E1A6F120EFE
:1011E0001D6FD20E1C6F120E1F6F840E1E6F120E1B
:1011F000216F380E206F110E236FED0E226F110E2E
:10120000256FA30E246F110E276F5A0E266F110E35
:10121000296F120E286F100E2B6FCC0E2A6F100E36
:101220002D6F870E2C6F100E2F6F420E2E6F0F0E2C
:10123000316F3069336FBD0E326F0F0E356F7C0E1C
:10124000346F0F0E376F3D0E366F0E0E396FFE0E78
:10125000386F0E0E3B6FC00E3A6F0E0E3D6F830E51
:101260003C6F0E0E3F6F470E3E6F0E0E416F0C0E21
:10127000406F0D0E436FD20E426F0D0E456F990EEB
:10128000446F0D0E476F610E466F0D0E496F2A0EAB
:10129000486F0C0E4B6FF40E4A6F0C0E4D6FBE0E66
:1012A0004C6F0C0E4F6F8A0E4E6F0C0E516F560E18
:1012B000506F0C0E536F230E526F0B0E556FF10EC5
:1012C000546F0B0E576FC00E566F01014D694C697C
:1012D000A20E4F6FC30E4E6F9A0E516F460E506F97
:1012E000960E536F320E526F920E556F3A0E546F28
:1012F0008E0E576F5D0E566F8A0E596F9A0E586F8D
:10130000860E5B6FF00E5A6F830E5D6F5F0E5C6F23
:101310007F0E5F6FE70E5E6F7C0E616F850E606FF4
:10132000790E636F3B0E626F760E656F070E646F0A
:10133000720E676FE80E666F6F0E696FDF0E686F73
:101340006C0E6B6FEA0E6A6F6A0E6D6F0A0E6C6F31
:10135000670E6F6F3C0E6E6F640E716F820E706F52
:10136000610E736FDA0E726F5F0E756F440E746FDD
:101370005C0E776FBF0E766F5A0E796F4C0E786FDA
:10138000570E7B6FE90E7A6F550E7D6F960E7C6F50
:10139000530E7F6F7E6F510E816F200E806F4E0E49
:1013A000836FFB0E826F4C0E856FE50E846F4A0EC5
:1013B000876FDC0E866F480E896FE20E886F460ECF
:1013C0008B6FF50E8A6F450E8D6F150E8C6F430E69
:1013D0008F6F420E8E6F410E916F7B0E906F3F0E9E
:1013E000936FC00E926F3E0E956F100E946F3C0E71
:1013F000976F6D0E966F3A0E996FD40E986F390EE7
:101400009B6F460E9A6F370E9D6FC20E9C6F360E05
:101410009F6F490E9E6F340EA16FDA0EA06F330ED0
:10142000A36F740EA26F320EA56F180EA46F300E4C
:10143000A76FC50EA66F2F0EA96F7B0EA86F2E0E7D
:10144000AB6F3A0EAA6F2D0EAD6F020EAC6F2B0E66
:10145000AF6FD10EAE6F2A0EB16FA90EB06F290E0D
:10146000B36F880EB26F280EB56F6F0EB46F270E74
:10147000B76F5E0EB66F260EB96F530EB86F250E9E
:10148000BB6F500EBA6F240EBD6F540EBC6F230E8F
:10149000BF6F5E0EBE6F220EC16F6F0EC06F210E4A
:1014A000C36F860EC26F200EC56FA30EC46F1F0ED2
:1014B000C76FC60EC66F1E0EC96FEF0EC86F1E0E29
:1014C000CB6FCA6F1D0ECD6F520ECC6F1C0ECF6F3F
:1014D0008C0ECE6F1B0ED16FCB0ED06F1B0ED36F49
:1014E0000F0ED26F1A0ED56F580ED46F190ED76F1C
:1014F000A50ED66F180ED96FF80ED86F180EDB6FC9
:101500004F0EDA6F170EDD6FAB0EDC6F170EDF6F4D
:101510000A0EDE6F160EE16F6F0EE06F150EE36FB1
:10152000D70EE26F150EE56F430EE46F140EE76FF2
:10153000B30EE66F140EE96F270EE86F130EEB6F14
:101540009F0EEA6F130EED6F1A0EEC6F120EEF6F17
:10155000990EEE6F120EF16F1B0EF06F110EF36FFE
:10156000A10EF26F110EF56F290EF46F100EF76FCA
:10157000B50EF66F100EF96F440EF86F0F0EFB6F7D
:10158000D60EFA6F0F0EFD6F6B0EFC6F0F0EFF6F16
:10159000030EFE6F0E0E0201016F9D0E006F0E0E08
:1015A000036F3A0E026F0D0E056FDA0E046F0D0E0B
:1015B000076F7C0E066F0D0E096F210E086F0C0E63
:1015C0000B6FC80E0A6F0C0E0D6F720E0C6F0C0EA7
:1015D0000F6F1E0E0E6F0B0E116FCC0E106F0B0ED9
:1015E000136F7C0E126F0B0E156F2E0E146F0A0EFA
:1015F000176FE30E166F0A0E196F990E186F0A0E09
:101600001B6F510E1A6F0A0E1D6F0B0E1C6F090E09
:101610001F6FC80E1E6F090E216F850E206F090EF9
:10162000236F450E226F090E256F060E246F080EDC
:10163000276FC90E266F080E296F8E0E286F080EB1
:101640002B6F540E2A6F080E2D6F1C0E2C6F070E79
:101650002F6FE50E2E6F070E316FAF0E306F070E36
:10166000336F7B0E326F070E356F490E346F070EE6
:10167000376F170E366F060E396FE70E386F060E8E
:101680003B6FB90E3A6F060E3D6F8B0E3C6F060E28
:101690003F6F5F0E3E6F060E416F340E406F060EB9
:1016A000436F0A0E426F050E456FE10E446F050E43
:1016B000476FB90E466F050E496F930E486F050EC2
:1016C0004B6F6D0E4A6F156A0001800E155C22E2A9
:1016D00001EE4CF0D8901534E926000EEA22EECF48
:1016E00005F0EFCF06F00630026E0530016E0232D3
:1016F0000132023201321F0E021601EE4CF0D89078
:101700001534E926000EEA2201C0EEFF02C0EFFF09
:10171000152ADAE31200040E03015B6F880E5A6F7C
:10172000040E5D6FA60E5C6F040E5F6FB60E5E6FEB
:10173000040E616FC60E606F040E636FD60E626F8B
:10174000040E656FE60E646F040E676FF60E666F2B
:10175000050E696F070E686F050E6B6F170E6A6FC7
:10176000050E6D6F280E6C6F050E6F6F390E6E6F64
:10177000050E716F4B0E706F050E736F5D0E726FFD
:10178000050E756F6E0E746F050E776F800E766F97
:10179000050E796F930E786F050E7B6FA50E7A6F2D
:1017A000050E7D6FB80E7C6F050E7F6FCB0E7E6FC2
:1017B000050E816FDF0E806F050E836FF20E826F54
:1017C000060E856F846F876F1A0E866F060E896FFF
:1017D0002E0E886F060E8B6F430E8A6F060E8D6F6E
:1017E000580E8C6F060E8F6F6D0E8E6F060E916FFA
:1017F000830E906F060E936F980E926F060E956F84
:10180000AE0E946F060E976FC40E966F060E996F0C
:10181000DB0E986F060E9B6FF20E9A6F070E9D6F90
:10182000090E9C6F070E9F6F210E9E6F070EA16F12
:10183000380EA06F070EA36F500EA26F070EA56F94
:10184000690EA46F070EA76F810EA66F070EA96F12
:101850009A0EA86F070EAB6FB40EAA6F070EAD6F8E
:10186000CD0EAC6F070EAF6FE70EAE6F080EB16F07
:10187000020EB06F080EB36F1D0EB26F080EB56F7B
:10188000380EB46F080EB76F530EB66F080EB96FEF
:101890006F0EB86F080EBB6F8B0EBA6F080EBD6F60
:1018A000A70EBC6F080EBF6FC40EBE6F080EC16FCF
:1018B000E10EC06F080EC36FC269090EC56F1D0E21
:1018C000C46F090EC76F3B0EC66F090EC96F5A0E63
:1018D000C86F090ECB6F790ECA6F090ECD6F990EC6
:1018E000CC6F090ECF6FB90ECE6F090ED16FD90E26
:1018F000D06F090ED36FFA0ED26F0A0ED56F1B0E82
:10190000D46F0A0ED76F3D0ED66F0A0ED96F5F0ED9
:10191000D86F0A0EDB6F820EDA6F0A0EDD6FA50E2E
:10192000DC6F0A0EDF6FC80EDE6F0A0EE16FEC0E81
:10193000E06F0B0EE36F110EE26F0B0EE56F360ECC
:10194000E46F0B0EE76F5B0EE66F0B0EE96F810E17
:10195000E86F0B0EEB6FA70EEA6F0B0EED6FCE0E5E
:10196000EC6F0B0EEF6FF50EEE6F0C0EF16F1D0EA0
:10197000F06F0C0EF36F460EF26F0C0EF56F6F0EDC
:10198000F46F0C0EF76F980EF66F0C0EF96FC20E17
:10199000F86F0C0EFB6FED0EFA6F0D0EFD6F180E4B
:1019A000FC6F0D0EFF6F430EFE6F0D0E0401016FF5
:1019B000700E006F0D0E036F9C0E026F0D0E056F03
:1019C000CA0E046F0D0E076FF80E066F0E0E096F2C
:1019D000260E086F0E0E0B6F550E0A6F0E0E0D6F52
:1019E000850E0C6F0E0E0F6FB60E0E6F0E0E116F72
:1019F000E70E106F0F0E136F180E126F0F0E156F8C
:101A00004B0E146F0F0E176F7E0E166F0F0E196FA1
:101A1000B10E186F0F0E1B6FE60E1A6F100E1D6FB2
:101A20001B0E1C6F100E1F6F500E1E6F100E216FBD
:101A3000870E206F100E236FBE0E226F100E256FC3
:101A4000F60E246F110E276F2E0E266F110E296FC2
:101A5000680E286F110E2B6FA20E2A6F110E2D6FBC
:101A6000DC0E2C6F120E2F6F180E2E6F120E316FB0
:101A7000540E306F120E336F910E326F120E356F9F
:101A8000CF0E346F130E376F0E0E366F130E396F85
:101A90004D0E386F130E3B6F8E0E3A6F130E3D6F67
:101AA000CF0E3C6F140E3F6F110E3E6F140E416F40
:101AB000540E406F140E436F980E426F140E456F14
:101AC000DC0E446F150E476F220E466F150E496FE0
:101AD000680E486F150E4B6FB00E4A6F150E4D6FA6
:101AE000F80E4C6F160E4F6F410E4E6F160E516F63
:101AF0008C0E506F160E536FD70E526F170E556F18
:101B0000230E546F170E576F700E566F00011200A0
:101B1000FB0E02014D6F1D0E4C6FFB0E4F6F260E1C
:101B20004E6FFB0E516F2F0E506FFB0E536F370E23
:101B3000526FFB0E556F400E546FFB0E576F490EE0
:101B4000566FFB0E596F520E586FFB0E5B6F5B0E9C
:101B50005A6FFB0E5D6F630E5C6FFB0E5F6F6C0E5A
:101B60005E6FFB0E616F750E606FFB0E636F7E0E16
:101B7000626FFB0E656F860E646FFB0E676F8F0ED4
:101B8000666FFB0E696F980E686FFB0E6B6FA10E90
:101B90006A6FFB0E6D6FAA0E6C6FFB0E6F6FB20E4D
:101BA0006E6FFB0E716FBB0E706FFB0E736FC40E0A
:101BB000726FFB0E756FCD0E746FFB0E776FD60EC6
:101BC000766FFB0E796FDE0E786FFB0E7B6FE70E84
:101BD0007A6FFB0E7D6FF00E7C6FFB0E7F6FF90E40
:101BE0007E6FFC0E816F020E806FFC0E836F0A0EFB
:101BF000826FFC0E856F130E846FFC0E876F1C0EB8
:101C0000866FFC0E896F250E886FFC0E8B6F2D0E74
:101C10008A6FFC0E8D6F360E8C6FFC0E8F6F3F0E31
:101C20008E6FFC0E916F480E906FFC0E936F510EED
:101C3000926FFC0E956F590E946FFC0E976F620EAB
:101C4000966FFC0E996F6B0E986FFC0E9B6F740E67
:101C50009A6FFC0E9D6F7D0E9C6FFC0E9F6F850E24
:101C60009E6FFC0EA16F8E0EA06FFC0EA36F970EE1
:101C7000A26FFC0EA56FA00EA46FFC0EA76FA90E9D
:101C8000A66FFC0EA96FB10EA86FFC0EAB6FBA0E5B
:101C9000AA6FFC0EAD6FC30EAC6FFC0EAF6FCC0E17
:101CA000AE6FFC0EB16FD40EB06FFC0EB36FDD0ED5
:101CB000B26FFC0EB56FE60EB46FFC0EB76FEF0E91
:101CC000B66FFC0EB96FF80EB86FFD0EBB6FBA6B36
:101CD000BD6F090EBC6FFD0EBF6F120EBE6FFD0E05
:101CE000C16F1B0EC06FFD0EC36F240EC26FFD0EC1
:101CF000C56F2C0EC46FFD0EC76F350EC66FFD0E7F
:101D0000C96F3E0EC86FFD0ECB6F470ECA6FFD0E3A
:101D1000CD6F500ECC6FFD0ECF6F580ECE6FFD0EF7
:101D2000D16F610ED06FFD0ED36F6A0ED26FFD0EB4
:101D3000D56F730ED46FFD0ED76F7B0ED66FFD0E71
:101D4000D96F840ED86FFD0EDB6F8D0EDA6FFD0E2E
:101D5000DD6F960EDC6FFD0EDF6F9F0EDE6FFD0EEA
:101D6000E16FA70EE06FFD0EE36FB00EE26FFD0EA8
:101D7000E56FB90EE46FFD0EE76FC20EE66FFD0E64
:101D8000E96FCB0EE86FFD0EEB6FD30EEA6FFD0E21
:101D9000ED6FDC0EEC6FFD0EEF6FE50EEE6FFD0EDE
:101DA000F16FEE0EF06FFD0EF36FF60EF26FFD0E9B
:101DB000F56FF469FE0EF76F080EF66FFE0EF96F01
:101DC000110EF86FFE0EFB6F1A0EFA6FFE0EFD6F0E
:101DD000220EFC6FFE0EFF6F2B0EFE6FFE0E030138
:101DE000016F340E006FFE0E036F3D0E026FFE0E8C
:101DF000056F460E046FFE0E076F4E0E066FFE0E49
:101E0000096F570E086FFE0E0B6F600E0A6FFE0E05
:101E10000D6F690E0C6FFE0E0F6F720E0E6FFE0EC1
:101E2000116F7A0E106FFE0E136F830E126FFE0E7F
:101E3000156F8C0E146FFE0E176F950E166FFE0E3B
:101E4000196F9D0E186FFE0E1B6FA60E1A6FFE0EF9
:101E50001D6FAF0E1C6FFE0E1F6FB80E1E6FFE0EB5
:101E6000216FC10E206FFE0E236FC90E226FFE0E72
:101E7000256FD20E246FFE0E276FDB0E266FFE0E2F
:101E8000296FE40E286FFE0E2B6FED0E2A6FFE0EEB
:101E90002D6FF50E2C6FFE0E2F6F2E6F3169070E12
:101EA000306F3369100E326F3569190E346F376930
:101EB000210E366F39692A0E386F3B69330E3A6F3F
:101EC0003D693C0E3C6F3F69440E3E6F41694D0ECB
:101ED000406F4369560E426F45695F0E446F476914
:101EE000680E466F4969700E486F4B69790E4A6FEC
:061EF00000011200FFD703
:020000040030CA
:0300010006160ED2
:020005008580F4
:060008000FC00FE00F40E5
:00000001FF
